:04000000B8EF0CF059
:1000080000C016F001C015F0F2A419D0010E1D149D
:10001800016E0150010A02E1818C01D0819C020E1F
:100028001D14016E0150020A02E1818E02D07F0E7A
:100038008116D10ED76E3A0ED66E4B80F29416C04A
:0800480000F015C001F01100E9
:1000500081CF03F00001D05305E0C00E0314026EFF
:10006000028803D0C00E0314026ED1C000F000322B
:10007000009E0032009E0032009E0032009E0F0E55
:10008000001602500010016E0F0ED115006E0250C6
:100090000012200E0110816E01C081FF200E0010A1
:1000A000816E00C081FF03C081FF9F0E0D6E0D2E7B
:0800B000FED700000000120061
:1000B8000001D06B060E016ECEC000F0015004E0C6
:1000C80000360090FF0FFBD70050800FD16FCC5146
:1000D800D127BADF020E0C6E8D0E0D6E0D2EFED7D7
:0A00E8000C2EFCD7000000001200EF
:1000F2000001CC6BCD6BCE6BCF6BDDDFCA6BCB6BF4
:10010200800ECB19006E800E005C02E1100ECA5DFB
:1001120025E2800ECB19006E800E4218005C02E1CF
:100122004150CA5D13E2010ED06FCAC000F0CBC0CD
:1001320001F0003600900136210E0024E96E000E17
:100142000120EA6EEECFD1F082DF05D0010ED06F32
:10015200200ED16F7CDFCA4BCB2BD2D7416A426AC9
:10016200CC6BCD6B010ECE6F000ECF6FA4DFCA6BCE
:10017200CB6B800ECB19006E800E005C02E1100E7C
:10018200CA5D08E2010ED06F200ED16F60DFCA4B4C
:10019200CB2BEFD7CC6BCD6B010ECE6F000ECF6F9A
:0401A2008ADF1200DE
:1001A6000001CC6BCD6BCE6BCF6B83DFC86BC96B9D
:1001B600800EC919006E800E005C02E1100EC85D4B
:1001C60008E2010ED06F200ED16F3FDFC84BC92B5E
:1001D600EFD7CC6BCD6B010ECE6F000ECF6F69DF04
:1001E600C86BC96B800EC919006E800E005C02E1F7
:1001F600100EC85D08E2010ED06F200ED16F25DF0C
:10020600C84BC92BEFD7CC6BCD6BCE6BCF6B51DF09
:0A021600446A456A416A426A120018
:100220000001C8510A0A16E1000E451802E1000E4D
:1002300044180EE1010E446E000E456E416A426A9A
:10024000CC6BCD6B010ECE6F000ECF6F35DF01D0C2
:1002500050DF31D041C000F042C001F000360090C4
:100260000136210E0024E16E000E0120E26EC8C0AE
:10027000E6FF000EE66E414A422A800E4218006EEA
:10028000800E005C02E1100E415C15E3000E451883
:1002900002E1000E44180EE1010E446E000E456EA0
:1002A000416A426ACC6BCD6B010ECE6F000ECF6FF0
:0802B00003DF01D01EDF120084
:1002B80010D075DF19D0C7C0C8F0AEDF15D014D084
:1002C800010ED06FC7C0D1F0BFDEC7C0C8F0A4DF31
:1002D8000BD00001C7510C0AECE0C7510A0AEBE049
:0A02E800C7510D0AECE0ECD712003C
:1002F2000001C56BC66B800EC619006E800E005CD5
:1003020002E1100EC55D16E2C551C325E96EC65164
:10031200C421EA6EEE50000A01E10CD0C551C3259A
:10032200E96EC651C421EA6EEECFC7F0C4DFC54BF9
:06033200C62BE1D712000A
:100338000134083609360450085E0550D8A0053C3B
:10034800095E003601360F0E0C6E01340836093688
:10035800045000A006D0085E0550D8A0053C095EF0
:1003680005D008260550D8B0053C092600360136C8
:100378000C2EEBD700B006D0045008260550D8B094
:08038800053C092600001200EB
:100390000B6A0A6A096A00500402F4CF09F0F3CF2D
:1003A00008F001500502F4CF0BF0F3CF0AF0005033
:1003B0000502F3500926F4500A22E86A0B22015084
:1003C0000402F3500926F4500A22E86A0B2208C0FE
:1003D00000F009C001F00AC002F00BC003F01200E7
:1003E0000001C46B0E0EC45D1DE20A0EC403F3CF00
:1003F00000F0F4CF01F0AA0E0024F66E1A0E0120D0
:10040000F76E000EF86E000E01BEFF0EF822090016
:10041000F5CF01F00150C31903E1C4C000F0120090
:0A042000C42BE0D7FF0E006E12009F
:10042A00150E0001BE6FB86BB96B800EB919006E5C
:10043A00800E005C02E10D0EB85DD8B081D0B8C064
:10044A0000F0B9C001F00A0E046E000E056E9BDFC3
:10045A00004A012A360E0024F66E1B0E0120F76EA2
:10046A00000EF86E000E01BEFF0EF8220900F5CF4D
:10047A0001F0000EB71902E10150B6195EE1010E52
:10048A00BC6F000EBD6FBA6BBB6B800EBB19006EE2
:10049A00800EB719005C02E1B651BA5D2FE2BA517B
:1004AA00B425E96EBB51B521EA6EB8C000F0B9C0F7
:1004BA0001F00A0E046E000E056E65DF020E0026BC
:1004CA00000E0122BA510026BB510122360E002429
:1004DA00F66E1B0E0120F76E000EF86E000E01BEBE
:1004EA00FF0EF8220900F5CF01F0EE50011803E0E3
:1004FA00BC6BBD6B03D0BA4BBB2BC7D7000EBD1963
:10050A0002E1010EBC1919E1B8C000F0B9C001F04E
:10051A000A0E046E000E056E36DF360E0024F66EE5
:10052A001B0E0120F76E000EF86E000E01BEFF0EC4
:10053A00F8220900F5CFBEF003D0B84BB92B75D716
:06054A00BEC000F012002B
:100550000450000A08E10550000A05E1FF0E006E94
:100560007F0E016E12000D6A096A086A01500010C0
:10057000D8B4000C015005180A6E0ABE0D1E0B6A95
:1005800005AE05D0041E051E042AD8B4052A01AE06
:1005900005D0001E011E002AD8B4012A0150051002
:1005A0000A6E0ABE10D0C8DE0BB020D00DAE000C13
:1005B000001E011E002AD8B4012A081E091E082A9E
:1005C000D8B4092A000C05AE0DD001BE07D00150E9
:1005D000096E0050086E016A006AE8D7016A006A75
:1005E000002A000C011E001E0B2ADDD7082AD8B4F1
:1005F000092A0450085CD8A4D9D70550095CD8A4AE
:10060000D5D7096A086A002AD8B4012A01AECED724
:060610000000FF0C1200C7
:10061600150E0001BE6FB86BB96B800EB919006E6E
:10062600800E005C02E10A0EB85DD8B081D0B8C079
:1006360000F0B9C001F00A0E046E000E056EA5DECC
:10064600004A012A3A0E0024F66E1C0E0120F76EAF
:10065600000EF86E000E01BEFF0EF8220900F5CF5F
:1006660001F0000EB71902E10150B6195EE1010E64
:10067600BC6F000EBD6FBA6BBB6B800EBB19006EF4
:10068600800EB719005C02E1B651BA5D2FE2BA518D
:10069600B425E96EBB51B521EA6EB8C000F0B9C009
:1006A60001F00A0E046E000E056E6FDE020E0026C5
:1006B600000E0122BA510026BB5101223A0E002437
:1006C600F66E1C0E0120F76E000EF86E000E01BECF
:1006D600FF0EF8220900F5CF01F0EE50011803E0F5
:1006E600BC6BBD6B03D0BA4BBB2BC7D7000EBD1975
:1006F60002E1010EBC1919E1B8C000F0B9C001F061
:100706000A0E046E000E056E40DE3A0E0024F66EEA
:100716001C0E0120F76E000EF86E000E01BEFF0ED5
:10072600F8220900F5CFBEF003D0B84BB92B75D728
:06073600BEC000F012003D
:10073C00150E0001BE6FB86BB96B800EB919006E47
:10074C00800E005C02E10E0EB85DD8B081D0B8C04E
:10075C0000F0B9C001F00A0E046E000E056E12DE38
:10076C00004A012AAA0E0024F66E1A0E0120F76E1A
:10077C00000EF86E000E01BEFF0EF8220900F5CF38
:10078C0001F0000EB71902E10150B6195EE1010E3D
:10079C00BC6F000EBD6FBA6BBB6B800EBB19006ECD
:1007AC00800EB719005C02E1B651BA5D2FE2BA5166
:1007BC00B425E96EBB51B521EA6EB8C000F0B9C0E2
:1007CC0001F00A0E046E000E056EDCDD020E002632
:1007DC00000E0122BA510026BB510122AA0E0024A0
:1007EC00F66E1A0E0120F76E000EF86E000E01BEAA
:1007FC00FF0EF8220900F5CF01F0EE50011803E0CE
:10080C00BC6BBD6B03D0BA4BBB2BC7D7000EBD194D
:10081C0002E1010EBC1919E1B8C000F0B9C001F039
:10082C000A0E046E000E056EADDDAA0E0024F66EE7
:10083C001A0E0120F76E000EF86E000E01BEFF0EB0
:10084C00F8220900F5CFBEF003D0B84BB92B75D701
:06085C00BEC000F0120016
:10086200150E0001BE6FB86BB96B800EB919006E20
:10087200800E005C02E10D0EB85DD8B081D0B8C028
:1008820000F0B9C001F00A0E046E000E056E7FDDA5
:10089200004A012AB80E0024F66E1B0E0120F76EE4
:1008A200000EF86E000E01BEFF0EF8220900F5CF11
:1008B20001F0000EB71902E10150B6195EE1010E16
:1008C200BC6F000EBD6FBA6BBB6B800EBB19006EA6
:1008D200800EB719005C02E1B651BA5D2FE2BA513F
:1008E200B425E96EBB51B521EA6EB8C000F0B9C0BB
:1008F20001F00A0E046E000E056E49DD020E00269E
:10090200000E0122BA510026BB510122B80E00246A
:10091200F66E1B0E0120F76E000EF86E000E01BE81
:10092200FF0EF8220900F5CF01F0EE50011803E0A6
:10093200BC6BBD6B03D0BA4BBB2BC7D7000EBD1926
:1009420002E1010EBC1919E1B8C000F0B9C001F012
:100952000A0E046E000E056E1ADDB80E0024F66E45
:100962001B0E0120F76E000EF86E000E01BEFF0E88
:10097200F8220900F5CFBEF003D0B84BB92B75D7DA
:06098200BEC000F01200EF
:10098800B4C004F0B5C005F004C0E9FF05C0EAFF33
:10099800EE5203E0044A052AF7D704C002F005C066
:1009A80003F0044A052AB6C000F0B7C001F0000100
:1009B800B64BB72B00C0E9FF01C0EAFF02C0E1FF58
:1009C80003C0E2FFEECFE6FF02C0E9FF03C0EAFF83
:1009D800EE5201E0E2D7B4C000F0B5C001F0120059
:1009E800B4C004F0B5C005F004C002F005C003F0BF
:1009F800044A052AB6C000F0B7C001F00001B64BA2
:100A0800B72B00C0E9FF01C0EAFF02C0E1FF03C045
:100A1800E2FFEECFE6FF02C0E9FF03C0EAFFEE52B5
:0E0A280001E0E2D7B4C000F0B5C001F012004A
:100A3600300E0001B45D33E3B451390830E37F6B07
:100A4600300EB45D006E00C083F0826B0A0E0002A9
:100A5600F3CF00F0F4CF01F0020E0026000E0122C3
:100A66003A0E0024F66E1C0E0120F76E000EF86E8C
:100A7600000E01BEFF0EF8220900F5CF00F0000EB1
:100A8600016E6CC004F06DC005F07FDC00C080F024
:100A960001C081F0010E1E6E030E1D121200610EC2
:100AA600B45D05E3B4517A0802E3200EB45F410E4B
:100AB600B45D34E3B4514D0831E3010E7F6F410E4E
:100AC600B45D006E00C083F0826B0A0E0002F3CFA5
:100AD60000F0F4CF01F0020E0026000E0122360EC1
:100AE6000024F66E1B0E0120F76E000EF86E000E47
:100AF60001BEFF0EF8220900F5CF00F0000E016ED0
:100B06006CC004F06DC005F040DC00C080F001C090
:100B160081F0010E1E6E030E1D1212004E0EB45D04
:100B260034E3B4515A0831E3020E7F6F4E0EB45DC2
:100B3600006E00C083F0826B0A0E0002F3CF00F055
:100B4600F4CF01F0020E0026000E0122B80E00249A
:100B5600F66E1B0E0120F76E000EF86E000E01BE3B
:100B6600FF0EF8220900F5CF00F0000E016E6CC0F2
:100B760004F06DC005F009DC00C080F001C081F012
:100B8600010E1E6E030E1D121200B4C0C3F025DC4A
:100B960000C0B5F0000E016EFF0E011802E1FF0E57
:100BA600001801E11200030E7F6FB5C083F0826B5F
:100BB6000A0EB503F3CF00F0F4CF01F0020E0026C3
:100BC600000E0122AA0E0024F66E1A0E0120F76E00
:100BD600000EF86E000E01BEFF0EF8220900F5CFDA
:100BE60000F0000E016E6CC004F06DC005F0C8EC9C
:100BF60001F000C080F001C081F0010E1E6E030EF0
:040C06001D121200A9
:100C0A00B20E0001B46FBC0EB56FDD0EB66FC30E27
:100C1A00B76FDE0EB86FDD0EB96FBC0EBA6FDD0EA0
:100C2A00BB6F200EBC6F560EBD6F310EBE6F2E0EFF
:100C3A00BF6F300EC06F0A0EC16FC26B2050000A20
:100C4A0008E1D3EC00F0B40EC36F000EC46F79EC68
:040C5A0001F0120093
:100C5E009DC0A9FF7F0EA616A69CA680A8CF01F068
:060C6E0001C000F01200BD
:100C74001E50000A01E0120000016E0EE96E000E23
:100C8400EA6E7E51E926D8B0EA2AEECF01F001C01F
:100C94009DF00150000A04E0100E7E5D01E204D0D4
:100CA400186A206AB0DF12009DC0B4F0C2DE7E2B49
:020CB40012002C
:100CB6000001A16BA26B9F6BA06B4950A05D02E186
:100CC60048509F5D43E29FC000F0A0C001F000368F
:100CD600009001364C0E0024E96E000E0120EA6EEB
:100CE600EECFACF0EECFADF09DC000F09EC001F0AF
:100CF6000C0E046E000E056EC8EC01F00A0E046EB2
:100D0600000E056E22DC800E0001AD19026E800E0B
:100D16000118025C02E10050AC5D09E2A40EA125B7
:100D2600E16E000EA221E26E010EE66E08D0A40E60
:100D3600A125E16E000EA221E26E030EE66EA14B26
:100D4600A22B020E9F27000EA023B7D7A40EB46FC6
:100D5600000EB56FA1C0B6F0A2C0B7F059DC00C056
:100D6600A3F00050150A0CE1A40EB46F000EB56F87
:100D7600A1C0B6F0A2C0B7F015EC02F000C0A3F017
:100D8600A351150A0BE1A40EB46F000EB56FA1C0F6
:100D9600B6F0A2C0B7F062DD00C0A3F0A351150AF9
:100DA6000BE1A40EB46F000EB56FA1C0B6F0A2C0E1
:0E0DB600B7F0C1DC00C0A3F0A3C000F0120033
:100DC400430E00019D6F610E9E6F6C0E9F6F6C0E43
:100DD400A06F200EA16F530EA26F690EA36F670E52
:100DE400A46F6E0EA56F2E0EA66F2E0EA76F2E0E7D
:100DF400A86F0A0EA96FAA6BD3EC00F09D0EC36F07
:0A0E0400000EC46F79EC01F012003B
:100E0E004E0E00019F6F470EA06F200EA16F430E76
:100E1E00A26F610EA36F6C0EA46F6C0EA56F200EE9
:100E2E00A66F530EA76F690EA86F670EA96F6E0E91
:100E3E00AA6F210EAB6F0A0EAC6FAD6BD3EC00F048
:100E4E009F0EC36F000EC46F79EC01F09DC0C3F00E
:0A0E5E009EC0C4F079EC01F0120010
:100E6800530E00019F6F650EA06F640EA16F690E8F
:100E7800A26F6E0EA36F670EA46F200EA56F430EB0
:100E8800A66F510EA76F2E0EA86F2E0EA96F2E0EED
:100E9800AA6F0A0EAB6FAC6B430EAD6F510EAE6FFF
:100EA800430EAF6F510EB06F440EB16F450EB26F67
:100EB800B36BD3EC00F09F0EC36F000EC46F79ECD8
:100EC80001F06E0EB46F000EB56FAD0EB66F000E6A
:100ED800B76F86DD6E0EB46F000EB56F9DC0B6F0AD
:100EE8009EC0B7F04DDD6E0EC36F000EC46F79EC77
:040EF80001F01200F3
:100EFC0081CF02F00001895305E0C00E0214016E8F
:100F0C00018803D0C00E0214016E01508A11006ECC
:100F1C00200E0010816E00C081FF02C081FF9F0E69
:0C0F2C000D6E0D2EFED70000000012001C
:100F380000018F6B8B6B8C6B8D6B8E6B010E896FC9
:100F4800000E8A6F020E485C016E000E4958026E50
:100F58008A51025C02E18951015C18E389C000F002
:100F68008AC001F00036009001364C0E0024D96E7C
:100F7800000E0120DA6EDE508D27DE508E238B4B5B
:100F88008C2B020E8927000E8A23DCD7800E006E78
:100F9800800E8C19005C02E18B51000847E28BC07F
:100FA80004F08CC005F08DC000F08EC001F0A8ECF4
:100FB80002F000C08DF001C08EF0800E026E800E2F
:100FC8000118025C02E10050320804E28DC019F0F9
:100FD8008EC01AF0010E485C036E000E4958046E6C
:100FE80003C000F004C001F00036009001364C0E3A
:100FF8000024E96E000E0120EA6EEECF03F0EECF7A
:1010080004F019C001F01AC002F00136019002364E
:101018000250045C02E10150035C07E319C09DF033
:101028001AC09EF044DE00C08FF04FD0010E485C1D
:10103800036E000E4958046E03C000F004C001F0AE
:101048000036009001364C0E0024E96E000E012097
:10105800EA6EEECF03F0EECF04F019C001F01AC02B
:1010680002F00136019002360450025C02E103509E
:10107800015C2BE2020E485C036E000E4958046EB8
:1010880003C000F004C001F00036009001364C0E99
:101098000024E96E000E0120EA6EEECF03F0EECFD9
:1010A80004F019C001F01AC002F0013601900236AE
:1010B8000250045C02E10150035C04E30001540E99
:1010C8008F6F03D00001450E8F6F8FC000F01200A4
:1010D80017061750000A03E1206A93DD186A120008
:1010E800080E1F14016E0150000A05E1FF0E1C5C7A
:1010F80001E21C2A77D0C80E1C5C1DE35FDE010EDE
:10110800186E040E206E7E6B1C6A896B8A6B800ECB
:101118008A19006E800E005C02E1070E895D0AE202
:101128006E0E8925E16E000E8A21E26EE66A894B11
:101138008A2BEDD757D00001896B8A6B800E8A19EC
:10114800006E800E005C02E1070E895D12E28B0ED4
:1011580089259B6F000E8A219C6F89C09DF07BDDDD
:101168009BC0E1FF9CC0E2FF00C0E6FF894B8A2BD1
:10117800E5D7896B8A6B800E8A19006E800E005C39
:1011880002E1070E895D0DE28B0E8925E96E000EDE
:101198008A21EA6EEE50000A01E103D0894B8A2BBE
:1011A800EAD7800E8A19006E800E005C02E1070EF5
:1011B800895D0CE3050E206E926B8B0E9D6F000E01
:1011C8009E6F21DEFF0E176E1C6A0CD0020E186E81
:1011D800030E206E8B0E9D6F000E9E6F41DE1C6A03
:0611E8007E6B44DD1200E5
:1011EE00080E1F14016E0150000A07E11C6A00016F
:0C11FE007E6B010E206E010E186E1200B8
:0E120A00570E0D6E0D2EFED7000000001200D4
:10121800A68489C0A9FF8AC0A8FF7F0EA616A69C2F
:10122800550EA76EAA0EA76EA682A6A201D0FDD75C
:021238001200A2
:10123A0000017F6B1E6A1B6A640E196E000E1A6E1D
:10124A001D6A176A140E4A6E640E6C6F000E6D6F7B
:02125A00120080
:10125C004B6A466A476A080ED56ED10ED76E3A0EA7
:0A126C00D66EA00EF26ED58E1200B1
:10127600FF0E926E936A946A816A946A826A050E78
:10128600C26E0E0EC16EBE0EC06E070EB46E12009A
:101296000900F5CFE6FF0006FBE10106F9E11200C1
:0612A600186A436A120001
:1012AC00030E0C6E550E0D6E0D2EFED70C2EFCD7AC
:1012BC000001856B866B800E8619006E800E005CBB
:1012CC0002E1030E855D07E2896B030E8A6F10DE67
:1012DC00854B862BF0D7896B020E8A6F09DED06B9B
:1012EC00280ED16F28EC00F0D06B100ED16F28ECCB
:1012FC0000F0D06B0E0ED16F28EC00F0D06B060E08
:10130C00D16F28EC00F0D06B010ED16F28EC00F0FF
:10131C00D06B020ED16F28EC00F0446A456A416A2A
:10132C00426A856B866B800E8619006E800E005C9F
:10133C0002E1100E855D0AE26E0E8525E16E000E4F
:0E134C008621E26EE66A854B862BEDD71200F5
:10135A0080501F18006E0C0E0014016E0150000A16
:10136A000DE04A50000808E24A064A50000A03E122
:0E137A000C0E80141F6E02D0140E4A6E12006C
:10138800C26A070EC012C08E85C000F000360090F9
:10139800003600900050C212C28033DFC282C2A25F
:1013A80001D0FDD7C4CF01F0006AC3500012000E6F
:0613B8000112C2901200B8
:1013BE000CD0829214D0828212D0432A140E435C37
:1013CE0002E3436A82720BD00AD01850000AF1E091
:1013DE001850010AF0E01850020AEFE0F5D712009B
:1013EE00060E00017E5D1EE2410E855D04E3855111
:1013FE005A0801E308D0300E855D04E385513908A3
:10140E0001E301D00FD06E0EE16E000EE26E7E5142
:10141E00E126D8B0E22A85C0E6FF7E2B85C0C7F054
:06142E005CEC01F012006D
:0A14340085C06CF086C06DF0120058
:10143E001E50010A02E1030E1D120ED10A0E00010A
:10144E008303F3CF02F0F4CF03F0010E0224006EFB
:10145E00000E0320016E3A0E0024F66E1C0E0120C3
:10146E00F76E000EF86E000E01BEFF0EF822090098
:10147E00F5CF85F0000E866F020E0224006E000E70
:10148E000320016E82510026000E01223A0E002426
:10149E00F66E1C0E0120F76E000EF86E000E01BEE9
:1014AE00FF0EF8220900F5CF00F0000E016E6CC0A1
:1014BE0004F06DC005F0C8EC01F000C087F001C06B
:1014CE0088F0DBD00A0E8303F3CF02F0F4CF03F0E3
:1014DE00010E0224006E000E0320016E360E002453
:1014EE00F66E1B0E0120F76E000EF86E000E01BE9A
:1014FE00FF0EF8220900F5CF85F0000E866F020E62
:10150E000224006E000E0320016E82510026000E92
:10151E000122360E0024F66E1B0E0120F76E000E11
:10152E00F86E000E01BEFF0EF8220900F5CF00F096
:10153E00000E016E6CC004F06DC005F0C8EC01F039
:10154E0000C087F001C088F098D00A0E8303F3CF55
:10155E0002F0F4CF03F0010E0224006E000E032001
:10156E00016EB80E0024F66E1B0E0120F76E000EF3
:10157E00F86E000E01BEFF0EF8220900F5CF85F0C1
:10158E00000E866F020E0224006E000E0320016E06
:10159E0082510026000E0122B80E0024F66E1B0E9C
:1015AE000120F76E000EF86E000E01BEFF0EF8223F
:1015BE000900F5CF00F0000E016E6CC004F06DC096
:1015CE0005F0C8EC01F000C087F001C088F055D0DE
:1015DE000A0E8303F3CF02F0F4CF03F0010E0224C0
:1015EE00006E000E0320016EAA0E0024F66E1A0E77
:1015FE000120F76E000EF86E000E01BEFF0EF822EF
:10160E000900F5CF85F0000E866F020E0224006EE3
:10161E00000E0320016E82510026000E0122AA0E3A
:10162E000024F66E1A0E0120F76E000EF86E000EF4
:10163E0001BEFF0EF8220900F5CF00F0000E016E7C
:10164E006CC004F06DC005F0C8EC01F000C087F06E
:10165E0001C088F012D011D000017F51000AD8B419
:10166E00EDD67F51010AD8B42DD77F51020AD8B4D6
:10167E006CD77F51030AACE0EED7010E805F000EEF
:10168E00815B000E811902E1000E80193FE134D01A
:10169E00822B800E006E800E8619005C02E1855151
:1016AE00825D11E36CC000F06DC001F0030E046E9C
:1016BE00000E056EC8EC01F000C080F001C081F094
:1016CE00030E1E6E06D06CC080F06DC081F0020E4F
:1016DE001E6EFC0E1D161AD087C080F088C081F0D9
:1016EE00010E1E6E030E1D1211D01E6AFC0E1D166B
:1016FE000DD0FC0E1D160AD01E50010AC9E01E5058
:0E170E00020AEAE01E50030AF0E0F3D71200D0
:10171C000001866BC9D0040E8515016E0150000ABC
:10172C0010E1010E486E000E496E006A016A4C0E03
:10173C000024E16E000E0120E26EE66AE66A010EFC
:10174C001B6EBED0040E8515016E0150000A26E1F9
:10175C00010E485C036E000E4958046E03C000F085
:10176C0004C001F00036009001364C0E0024026ECD
:10177C00000E0120036E02C0E9FF03C0EAFFEECFAA
:10178C0000F0EECF01F0004A012A02C0E1FF03C0D5
:10179C00E2FF00C0E6FF01C0E6FF23D0484A492A19
:1017AC00000E495C02E1100E485C04E31B6A86C023
:1017BC0000F01200010E485C036E000E4958046ED6
:1017CC0003C000F004C001F00036009001364C0E4E
:1017DC000024E16E000E0120E26EE66AE66A020E5B
:1017EC001B6E6ED0040E8515016E0150000A24E1AB
:1017FC00484A492A000E495C02E1100E485C04E399
:10180C001B6A86C000F01200010E485C036E000ECD
:10181C004958046E03C000F004C001F0003600907B
:10182C0001364C0E0024E16E000E0120E26EE66AD9
:10183C00E66A010E1B6E36D0010E485C036E000E7C
:10184C004958046E03C000F004C001F0003600904B
:10185C0001364C0E0024026E000E0120036E02C0F5
:10186C00E9FF03C0EAFFEECF00F0EECF01F0004A33
:10187C00012A02C0E1FF03C0E2FF00C0E6FF01C085
:10188C00E6FF9CEC07F000C086F00050150A05E15D
:10189C00210E0001866F1B6A05D000018651000ADB
:1018AC0001E01B6A0DD00CD01B50000AD8B433D702
:1018BC001B50010AD8B446D71B50020A93E0F3D749
:0618CC0086C000F01200CE
:1018D2003AD08CDC4BD007DC49D0080E1F14016EC5
:1018E2000150080A1FE1206A1C6A05EC06F0186A1A
:1018F200856B866B800E8619006E800E005C02E19D
:10190200070E855D0FE285C089F06E0E8525E96EB2
:10191200000E8621EA6EEECF8AF07DDC0001854B57
:10192200862BE8D723D03AEC06F020D0080E1F14FD
:10193200016E0150000A02E1020E206E17D06CEC1B
:1019420008F014D013D02050000AC3E02050010A3E
:10195200C2E02050020AC1E02050030AE4E0205015
:0E196200040AE4E02050050AEAE0ECD7120087
:101970000D0E0B6E2D0E0C6ED70E0D6E0D2EFED7AE
:101980000C2EFCD70B2EFAD700000000206A1D6A2F
:1019900072DC8CDC88DC62DC50DC80CF1FF09C0EBB
:1019A0000C6ED70E0D6E0D2EFED70C2EFCD705EC4F
:1019B00006F04BA05DD04B90464A472A0A0E046EB3
:1019C000000E056E46C000F047C001F0A8EC02F022
:1019D00008C000F009C001F0000E011802E1000E7D
:1019E000001801E14B82800E4718006E800E070A36
:1019F000005C02E1D00E465C02E3466A476AADDC59
:101A00002DD01DDD35D0040E1F14016E0150000ACB
:101A100002E11D8002D0FE0E1D161FC085F07EDE85
:101A200000C084F00050000A04E084C0C7F05CEC01
:101A300001F01ED0040E1F14016E0150000A02E1D5
:101A40001D8002D0FE0E1D161FC085F067DE00C08F
:101A500084F000C085F0CBDC0BD00AD02050030A04
:101A6000D0E02050000ACFE02050040AE3E0F5D790
:101A70004BA219D04B92A3DC0001856B85DC00C022
:101A800085F001C086F0000186338533869F86335A
:101A90008533869F86338533869F320E8527000ED9
:0A1AA0008623C8DC16DF85D7FFD7C8
:101AAA002E0601030103010300002C0603030101B2
:101ABA00030300003A0603030301010100003F0685
:101ACA0001010303010100002706010303030301C7
:101ADA0000002D060301010101030000280503018E
:101AEA0003030100000029060301030301030000A8
:101AFA002F0503010103010000003D050301010157
:101B0A00030000002B050103010301000000220667
:101B1A00010301010301000078040301010300002D
:0C1B2A000000400601030301030100005D
:101B3600410201030000000000004204030101010C
:101B460000000000430403010301000000004403F9
:101B56000301010000000000450101000000000033
:101B660000004604010103010000000047030303CF
:101B7600010000000000480401010101000000000E
:101B8600490201010000000000004A0401030303AA
:101B9600000000004B0303010300000000004C049A
:101BA60001030101000000004D02030300000000D4
:021BB60000002D
:101BB8004E0203010000000000004F03030303006E
:101BC800000000005004010303010000000051045C
:101BD8000303010300000000520301030100000099
:101BE800000053030101010000000000540103003C
:101BF8000000000000005503010103000000000080
:101C0800560401010103000000005703010303000B
:101C180000000000580403010103000000005904FB
:101C280003010303000000005A040303010100003C
:021C38000000AA
:101C3A003005030303030300000031050103030316
:101C4A00030000003205010103030300000033050D
:101C5A000101010303000000340501010101030031
:101C6A0000003505010101010100000036050301EC
:101C7A000101010000003705030301010100000012
:101C8A0038050303030101000000390503030303B8
:041C9A000100000045
:0E1C9E00536564696E672043512E2E2E0A0096
:071CAC004351435144450080
:0F1CB3004E472043616C6C205369676E210A0015
:0F1CC200B2BCDDC3DEDDBCDD2056312E300A00A2
:020000040030CA
:0E000000240E1F1EFF8381FF0FC00FE00F4074
:00000001FF
